:0200000480007A
:100000006F000005732F2034930F80006308FF03F7
:10001000930F90006304FF03930FB0006300FF038E
:10002000130F000063040F0067000F00732F2034CC
:1000300063540F006F00400093E19153171F0000BD
:1000400023223FFC171F000023200FFC6FF01FFF2F
:100050009300000013010000930100001302000050
:100060009302000013030000930300001304000038
:100070009304000013050000930500001306000020
:100080009306000013070000930700001308000008
:10009000930800001309000093090000130A0000F0
:1000A000930A0000130B0000930B0000130C0000D8
:1000B000930C0000130D0000930D0000130E0000C0
:1000C000930E0000130F0000930F0000732540F102
:1000D0006310050097020000938202017390523072
:1000E000735044749702000093820201739052305F
:1000F00073500018970200009382020273905230EE
:10010000B70200809382F2FF7390023B9302F001EA
:100110007390023A7350403097020000938242017C
:100120007390523073502030735030309301000080
:1001300097020000938242ED739052301305100035
:100140001315F501634C05000F00F00F930110002B
:100150009308D0051305000073000000930200000F
:10016000638A020073905210B7B20000938292101B
:100170007390223073500030372500007320053013
:100180007350300097020000938242017390123442
:10019000732540F1730020309301200017250000E3
:1001A000130545E607350500531505E293031000D6
:1001B000631275109301300017250000130505E543
:1001C00007350500531505E2930320006314750EEF
:1001D00093014000172500001305C5E3073505000E
:1001E000531505E2930340006316750C930150000C
:1001F00017250000130585E207350500531505E2B4
:10020000930380006318750A9301600017250000AE
:10021000130545E107350500531505E29303000179
:10022000631A75089301700017250000130505E097
:1002300007350500531505E293030002631C75069C
:1002400093018000172500001305C5DE0735050062
:10025000531505E293030004631E75049301900097
:1002600017250000130585DD07350500531505E248
:1002700093030008631075049301A0001725000084
:10028000130545DC07350500531505E293030010FF
:10029000631275029301B00017250000130505DBFA
:1002A00007350500531505E293030020631475001C
:1002B000631030020F00F00F638001009391110072
:1002C00093E111009308D00513850100730000002D
:1002D0000F00F00F930110009308D00513050000E4
:1002E00073000000731000C0000000000000000058
:0C02F00000000000000000000000000002
:1010000000000000000000000000000000000000E0
:1010100000000000000000000000000000000000D0
:1010200000000000000000000000000000000000C0
:1010300000000000000000000000000000000000B0
:081040000000000000000000A8
:10200000000000000000F0FF000000000000F0BF32
:10201000FFFFFFFFFFFF0F800000000000000080B7
:102020000000000000000000FFFFFFFFFFFF0F00A7
:10203000000000000000F03F000000000000F07F02
:10204000010000000000F07F000000000000F87FA9
:040000058000000077
:00000001FF
